:0300000002000EED
:03000300020028D0
:20000B0002001F758165D2AFD2A912002B80FE12001B80FB758CDC758A00050832050832A0
:20002B00E4F511747075F017F55485F055746475F000F54A85F04B745A75F000C0E0C0F099
:20004B00746475F000C0E0C0F01219831581158115811581120FEA1219B9748075F025C0D5
:20006B00E0C0F01219BC1581158179DF7A1C89828A83E493A3F5F0E493C0F0C0E01219DFFC
:20008B00158115811206BF1208081207231206941205B61203DB1204B11202351202A212B3
:2000AB0002E712091D120CB9120CF01210D4120ED412114F1212081216E01205870200926D
:2000CB00227F09121B80E4F5F078FD121B74F608A6F0121A0BC0E0C0F01219F3158115817A
:2000EB0078FC121B74F67B0D7C00121C80701902012E78FD121B74E60886F0121C3D18F68B
:20010B0008A6F0121C4680CA78FD121B74E60886F079F6121B79121B9678FC121B74E6F734
:20012B000200FD78FD121B74E60886F079F6121B79121B96E4F778FD121B74E60886F07B93
:20014B00007C00121C77700302015D74FFF5F002017079F6121B79E98AF0C0E0C0F0121AE1
:20016B001B158115817FF7021B8F05810581058105810581E4F5F078FD121B74F608A6F0FA
:20018B0078FD121B74E60886F07B027C00121C5770190201E178FD121B74E60886F0121C47
:2001AB003D18F608A6F0121C4680D578FD121B74E60886F079FA121B79121B96C001C002A9
:2001CB00121A0BC0E0C0F01219F315811581D007D000F60201A078FD121B74E60886F07910
:2001EB00FA121B79121B96E4F7E4F5F079FA121B79121B96E7C39430121BA67B04121B9D87
:20020B00121C1EC0E0C0F0740175F00079F8121B79121B96E7C39430D004D0034BC5F04C22
:20022B00C5F0121BA67FFB021B8FE51575F0007B697C00121C7770030202A1742275F01D71
:20024B00C0E0C0F01219DF15811581E4C0E0C0E012086015811581740475F000C0E0C0F016
:20026B001200CC7B647C00121BAFC0E0C0F0121A801581158115811581740475F000C0E08D
:20028B00C0F0121A6015811581F55485F055F55285F0531206BF22E511540875F0007B009E
:2002AB007C00121C8070030202E6E5528553F0121C46F55285F053121C3DE5528553F07B45
:2002CB00007C00121C9170030202E6E5548555F0F55285F053E5114404F51122E5161516DD
:2002EB00E51675F0007B007C00121C9170030203DA7464F516748575F000C0E0C0F0121ACE
:20030B009215811581C0E0C0F0E4C0E0C0E0121A5115811581D004D003121C77602B748329
:20032B0075F000C0E0C0F0121A9215811581C0E0C0F0740175F000C0E0C0F0121A51158186
:20034B001581D004D003121C7745F0700302036BE5114408F511742C75F001F54A85F04B4B
:20036B00748575F000C0E0C0F0121A9215811581C0E0C0F0740275F000C0E0C0F0121A51E2
:20038B0015811581D004D003121C77602B748375F000C0E0C0F0121A9215811581C0E0C059
:2003AB00F0740375F000C0E0C0F0121A5115811581D004D003121C7745F070030203DAE5B5
:2003CB001154F7F511746475F000F54A85F04B22E51575F0007B747C00121C77700302046A
:2003EB00B0742FF515743B75F01DC0E0C0F01219DF15811581748E75F000C0E0C0F0E4C083
:20040B00E0C0F01208111581158115811581748475F000C0E0C0F0120175121BA6C0E0C056
:20042B00F01208111581158115811581743A75F000C0E0C0F01219F315811581748275F036
:20044B0000C0E0C0F0120175121BA6C0E0C0F01208111581158115811581743A75F000C040
:20046B00E0C0F01219F315811581748075F000C0E0C0F0120175121BA6C0E0C0F012081118
:20048B001581158115811581748E75F000C0E0C0F07480C0E0C0F012081115811581158111
:2004AB0015811206BF22E51575F0007B647C00121C777003020586742FF515744875F01D58
:2004CB00C0E0C0F01219DF15811581748E75F000C0E0C0F0E4C0E0C0F01208111581158149
:2004EB0015811581748675F000C0E0C0F0120175121BA6C0E0C0F01208111581158115817E
:20050B001581742F75F000C0E0C0F01219F315811581748875F000C0E0C0F0120175121B32
:20052B00A6C0E0C0F01208111581158115811581742F75F000C0E0C0F01219F31581158195
:20054B00748C75F000C0E0C0F0120175121BA6C0E0C0F01208111581158115811581748EAB
:20056B0075F000C0E0C0F07480C0E0C0F012081115811581158115811206BF22E51575F09C
:20058B00007B0D7C00121C7770030205B579DF7A1C89828A83E493A3F5F0E493C0F0C0E0AC
:2005AB001219DF158115811206BF22E51575F0007B2F7C00121C777003020693745575F09B
:2005CB001DC0E0C0F0748775F000C0E0C0F0121A9215811581C0E0C0F0748975F000C0E0B7
:2005EB00C0F0121A9215811581C0E0C0F0748D75F000C0E0C0F0121A9215811581C0E0C006
:20060B00F0740475F00012173F7FF8121B80746675F01DC0E0C0F0748575F000C0E0C0F01C
:20062B00121A9215811581C0E0C0F0748375F000C0E0C0F0121A9215811581C0E0C0F0741B
:20064B008175F000C0E0C0F0121A9215811581C0E0C0F0740475F00012173F7FF8121B80B6
:20066B00120790747675F01DC0E0C0F0741775F000C0E0C0F0740275F00012173F158115DC
:20068B0081158115811206BF22E598540175F0007B007C00121C8070030206BA121A0BC0A1
:2006AB00E0C0F01219F315811581F5150206BE74FFF5152279E17A1C89828A83E493A3F5CF
:2006CB00F0E493C0F0C0E01219DF158115812205810581E4F5F078FD121B74F608A6F07809
:2006EB00FD121B74E60886F078F9121B748603088604121C57701902071E78FD121B74E68F
:20070B000886F0121C3D18F608A6F0121C4680CF020705158115812212072902075FE5503B
:20072B008551F0121C3DF55085F051121C46E5508551F0AB4AAC4B121C9A700302075EE491
:20074B00F5F0F55085F051E5114440F511C2B47405F51422E511544075F0007B007C00120C
:20076B001C80700302078FE5141514E51475F0007B007C00121C77700302078FD2B4E51124
:20078B0054BFF51122058105810581C2B5C2B4E4F5F078FC121B74F608A6F0121B2778FE58
:2007AB00121B74F67B007C00121C8070190207EB78FC121B74E60886F0121C3D18F608A6D5
:2007CB00F0121C4680D578FC121B74E60886F079177A00121B9678FE121B74E6F70207BB57
:2007EB0078FC121B74E60886F079177A00121B96E4F7D2B5D2B415811581158122308DFD22
:20080B00C28D438CDC220581058178F7121B74E6121BA678FD121B74F608A6F018E60886A6
:20082B00F07B087C00121C1E18F608A6F018E60886F078F9121B744608080808F608A6F03E
:20084B0018E60886F0C0E0C0F0121AC015811581158115812278FB121B74E6F513A2E09245
:20086B009020E106D291C2928004D292C291002205810581740175F000795A7A00121B96CC
:20088B00E775F00078FD121B74F608A6F018E60886F07B087C00121C1E18F608A6F0E4F50B
:2008AB00F0795A7A00121B9678FD121B74E60886F04715811581227401255AF55AE4355B67
:2008CB00F55BE4355CF55C221208C2740275F000795A7A00121B96E775F000C0E0C0F01260
:2008EB0008601581158112087B2278FB121B74E675F0007B047C00121C2CF62430C5F034BB
:20090B0000C5F02278FB121B74E6540F2430121BA622E511540475F0007B007C00121C80F7
:20092B007003020C7A1207901208D3C0E0C0F0748775F000C0E0C0F0121A9215811581C071
:20094B00E0C0F01208F515811581121BA6C0E0C0F0121A7215811581158115811208D3C0FB
:20096B00E0C0F0748775F000C0E0C0F0121A9215811581C0E0C0F012090F15811581121B6F
:20098B00A6C0E0C0F0121A7215811581158115811208D3C0E0C0F0748975F000C0E0C0F071
:2009AB00121A9215811581C0E0C0F01208F515811581121BA6C0E0C0F0121A7215811581CA
:2009CB00158115811208D3C0E0C0F0748975F000C0E0C0F0121A9215811581C0E0C0F012A5
:2009EB00090F15811581121BA6C0E0C0F0121A7215811581158115811208D3C0E0C0F074DE
:200A0B008D75F000C0E0C0F0121A9215811581C0E0C0F01208F515811581121BA6C0E0C0E1
:200A2B00F0121A7215811581158115811208D3C0E0C0F0748D75F000C0E0C0F0121A9215FF
:200A4B00811581C0E0C0F012090F15811581121BA6C0E0C0F0121A721581158115811581B5
:200A6B001208D3C0E0C0F0748575F000C0E0C0F0121A9215811581C0E0C0F01208F51581A1
:200A8B001581121BA6C0E0C0F0121A7215811581158115811208D3C0E0C0F0748575F00001
:200AAB00C0E0C0F0121A9215811581C0E0C0F012090F15811581121BA6C0E0C0F0121A728A
:200ACB0015811581158115811208D3C0E0C0F0748375F000C0E0C0F0121A9215811581C020
:200AEB00E0C0F01208F515811581121BA6C0E0C0F0121A7215811581158115811208D3C05A
:200B0B00E0C0F0748375F000C0E0C0F0121A9215811581C0E0C0F012090F15811581121BD1
:200B2B00A6C0E0C0F0121A7215811581158115811208D3C0E0C0F0748175F000C0E0C0F0D7
:200B4B00121A9215811581C0E0C0F01208F515811581121BA6C0E0C0F0121A721581158128
:200B6B00158115811208D3C0E0C0F0748175F000C0E0C0F0121A9215811581C0E0C0F0120B
:200B8B00090F15811581121BA6C0E0C0F0121A721581158115811581E4F5F0F55885F05909
:200BAB00E5588559F079177A00121B96E775F0007B007C00121C807015020C02E5588559B1
:200BCB00F0121C3DF55885F059121C4680D21208D3C0E0C0F0E5588559F079177A00121B4F
:200BEB0096E775F000C0E0C0F0121A721581158115811581020BC71208D3C0E0C0F0E4C00D
:200C0B00E0C0E0121A721581158115811581E51154FBF511E54E854FF0121C3DF54E85F0EE
:200C2B004F120C7BE4C0E0C0E012086015811581740675F000C0E0C0F0E54E854FF0C0E031
:200C4B00C0F0121A801581158115811581747975F01DC0E0C0F0E54E854FF0C0E0C0F0745B
:200C6B000275F00012173F158115811581158122E54E854FF07B887C13121C9A7003020C4E
:200C8B00B8E51154F7F511746475F000F54A85F04B743C75F000C0E0C0F074FFF5F0C0E0B1
:200CAB00C0F0121A72158115811581158122E51575F0007B727C00121C777003020CEF7410
:200CCB007C75F01DC0E0C0F0E54E854FF0C0E0C0F0740275F00012173F158115811581155A
:200CEB00811206BF22E51575F0007B737C00121C777003020E81E4C0E0C0E01208601581C9
:200D0B001581749275F01DC0E0C0F0E4C0E0C0E0121A5115811581C0E0C0F0740175F00063
:200D2B00C0E0C0F0121A5115811581C0E0C0F0740375F00012173F7FFA121B80E4C0E0C0B1
:200D4B00E0120175121BA6C0E0C0F0121A721581158115811581743A75F000C0E0C0F01292
:200D6B0019F315811581740175F000C0E0C0F0120175121BA6C0E0C0F0121A721581158191
:200D8B001581158174A575F01DC0E0C0F0740275F000C0E0C0F0121A5115811581C0E0C0FD
:200DAB00F0740375F000C0E0C0F0121A5115811581C0E0C0F0740375F00012173F7FFA1244
:200DCB001B80740275F000C0E0C0F0120175121BA6C0E0C0F0121A721581158115811581A1
:200DEB00743A75F000C0E0C0F01219F315811581740375F000C0E0C0F0120175121BA6C0F4
:200E0B00E0C0F0121A72158115811581158174B875F01DC0E0C0F0E4C0E0C0E0121A51158D
:200E2B00811581C0E0C0F0740175F000C0E0C0F0121A5115811581C0E0C0F0740275F00042
:200E4B00C0E0C0F0121A5115811581C0E0C0F0740375F000C0E0C0F0121A5115811581C0A9
:200E6B00E0C0F0740575F00012173F7FF6121B80120E821206BF22E4C0E0C0E0121A51151E
:200E8B008115817B997C00121C777003020EB7743C75F000C0E0C0F07401C0E0C0F0121A6B
:200EAB00721581158115811581020ED3743C75F000C0E0C0F074FFF5F0C0E0C0F0121A72CF
:200ECB00158115811581158122E51575F0007B3D7C00121C777003020FE9E4C0E0C0E012B2
:200EEB0008601581158174CE75F01DC0E0C0F0E4C0E0C0E0121A5115811581C0E0C0F074AE
:200F0B000175F000C0E0C0F0121A5115811581C0E0C0F0740375F00012173F7FFA121B80AD
:200F2B0074E075F01DC0E0C0F0740275F000C0E0C0F0121A5115811581C0E0C0F074037570
:200F4B00F000C0E0C0F0121A5115811581C0E0C0F0740375F00012173F7FFA121B8074F27D
:200F6B0075F01DC0E0C0F0740475F000C0E0C0F0121A60158115817B647C00121BC3C0E0C4
:200F8B00C0F0740275F00012173F1581158115811581743C75F000C0E0C0F0121A51158183
:200FAB0015817B017C00121C777003020FD1741075F01EC0E0C0F0740175F00012173F15F0
:200FCB00811581020FE6741975F01EC0E0C0F0740175F00012173F158115811206BF22E44D
:200FEB00C0E0C0E012086015811581740475F000C0E0C0F0121A6015811581F55485F05508
:20100B00F55285F053740675F000C0E0C0F0121A6015811581F54E85F04F746075F000C0CF
:20102B00E0C0F0742E75F000C0E0C0F01219831581158115811581745D75F000C0E0C0F032
:20104B00E54E854FF0C0E0C0F01219831581158115811581745D75F000C0E0C0F074607569
:20106B00F000C0E0C0F01218D51581158115811581745D75F000C0E0C0F0746475F000C04B
:20108B00E0C0F01219831581158115811581746375F000C0E0C0F0745D75F000C0E0C0F09D
:2010AB001218941581158115811581745A75F000C0E0C0F0746375F000C0E0C0F01219468F
:2010CB00158115811581158122E51575F0007B6E7C00121C77700302114E742075F01EC077
:2010EB00E0C0F01219DF15811581121A0B7B797C00121C77700302114BE51154F7F511E4D7
:20110B00F5F0F54E85F04F740675F000C0E0C0F0E4C0E0C0F0121A80158115811581158171
:20112B00745A75F000C0E0C0F0746475F000C0E0C0F01219831581158115811581121596D1
:20114B001206BF22E51575F0007B637C00121C777003021207743375F01EC0E0C0F074872A
:20116B0075F000C0E0C0F0121A9215811581C0E0C0F0748975F000C0E0C0F0121A9215816F
:20118B001581C0E0C0F0748D75F000C0E0C0F0121A9215811581C0E0C0F0740475F000127F
:2011AB00173F7FF8121B80744575F01EC0E0C0F0748575F000C0E0C0F0121A921581158186
:2011CB00C0E0C0F0748375F000C0E0C0F0121A9215811581C0E0C0F0748175F000C0E0C014
:2011EB00F0121A9215811581C0E0C0F0740475F00012173F7FF8121B801206BF22E51575E9
:20120B00F0007B617C00121C777003021324121656745D75F000C0E0C0F0740175F000C08C
:20122B00E0C0F01219831581158115811581745A75F000C0E0C0F0745D75F000C0E0C0F004
:20124B001218A71581158115811581745D75F000C0E0C0F0745A75F000C0E0C0F0121946E0
:20126B001581158115811581745A75F000C0E0C0F0746475F000C0E0C0F0121983158115A2
:20128B008115811581745D75F000C0E0C0F0745A75F000C0E0C0F01219611581158115813F
:2012AB0015817B007C00121C677003021321E4F5F0F55885F059E5588559F07B2E7C001232
:2012CB001C8A701502130AE5588559F0121C3DF55885F059121C4680DDE5588559F07917BC
:2012EB007A00121B96C001C0021208D3C0E0C0F0121A5115811581D007D000F60212D2E5D5
:20130B00588559F079177A00121B96E4F712132512154E0212901206BF22740D75F000C0F2
:20132B00E0C0F012158415811581740A75F000C0E0C0F012158415811581745575F01EC025
:20134B00E0C0F0E4F5F079177A00121B96E775F000C0E0C0F0740179177A00121B96E77522
:20136B00F000C0E0C0F0740279177A00121B96E775F000C0E0C0F0740379177A00121B96FF
:20138B00E775F000C0E0C0F0740479177A00121B96E775F000C0E0C0F0740579177A001230
:2013AB001B96E775F000C0E0C0F0740712173F7FF2121B80746475F01EC0E0C0F07406753A
:2013CB00F00079177A00121B96E775F000C0E0C0F0740779177A00121B96E775F000C0E075
:2013EB00C0F0740879177A00121B96E775F000C0E0C0F0740979177A00121B96E775F000B7
:20140B00C0E0C0F0740A79177A00121B96E775F000C0E0C0F0740B79177A00121B96E775E2
:20142B00F000C0E0C0F0740712173F7FF2121B80E4F5F0F55885F059E5588559F07B187C62
:20144B0000121C8A70170214D2E5588559F02403C5F03400C5F0F55885F05980DB747475B7
:20146B00F01EC0E0C0F0E5588559F0240DC5F03400C5F079177A00121B96E775F000C0E070
:20148B00C0F0E5588559F0240EC5F03400C5F079177A00121B96E775F000C0E0C0F0E55810
:2014AB008559F0240FC5F03400C5F079177A00121B96E775F000C0E0C0F0740412173F7FBA
:2014CB00F8121B80021454747C75F01EC0E0C0F0742575F00079177A00121B96E775F00018
:2014EB00C0E0C0F0742679177A00121B96E775F000C0E0C0F0742779177A00121B96E775CA
:20150B00F000C0E0C0F0742879177A00121B96E775F000C0E0C0F0742979177A00121B9611
:20152B00E775F000C0E0C0F0742A79177A00121B96E775F000C0E0C0F0740712173F7FF2A9
:20154B00021B8F0581121B207B137C00121C77700302158178FE121B74E6121BA67B1112D9
:20156B001B9D121C807003021581121B2078FE121B74F602155F15812278FB121B74E6F578
:20158B00133099FDC299E513F59922748A75F01EC0E0C0F01219DF15811581741775F0006D
:2015AB00C0E0C0F0743275F000C0E0C0F0121B321581158115811581E4C0E0C0E012086020
:2015CB0015811581E4F5F0F55885F059E5588559F079177A00121B96E775F0007B007C00D5
:2015EB00121C807015021636E5588559F0121C3DF55885F059121C4680D2E5588559F024D9
:20160B0008C5F03400C0F0C0E0E5588559F079177A00121B96E775F000C0E0C0F0121A726C
:20162B0015811581158115810215F3E5588559F02408C5F03400C0F0C0E0E4C0E0C0E01297
:20164B001A721581158115811581220581740D75F000C0E0C0F012158415811581740A75F3
:20166B00F000C0E0C0F012158415811581E4C0E0C0E012086015811581E4F5F0F55885F0F3
:20168B0059E5588559F02408C5F03400C0F0C0E0121A511581158178FE121B74F67B007CC9
:2016AB0000121C8070150216DDE5588559F0121C3DF55885F059121C4680C678FE121B7495
:2016CB00E6121BA6C0E0C0F01219F3158115810216B4158122E4C0E0C0E0120860158115DF
:2016EB0081743C75F000C0E0C0F0121A51158115817B017C00121C77700302173EE5B05400
:20170B000475F0007B007C00121C77700302172EE5114408F511742C75F001F54A85F04BB2
:20172B0002173EE51154F7F511746475F000F54A85F04B2223F42581F8868208868308E4E8
:20174B00FEFF93700122B42555A3E493B42D06430780A3E493B4300343074024D0B40A0025
:20176B00500CCE75F00AA42EFEA3E49380EDE493B46413E60886F030F708430720121C4D54
:20178B00A6F018F68003B4750543070A801CB478054307108014B46F0B430708800C1219A3
:2017AB00F9A3809BB462624307027A00C004C005C006C007AB0753031F7C00E60886F012FA
:2017CB001BEBA6F018F6EDD007D006D005D0042430B43A0040022407C0E00AE645F070CC61
:2017EB00A902EF30E506742D1219F90A121875D0E01219F9D9F90808EF30E7A5EAC39E50BF
:20180B00A074201219F90A80F3B4630BAA01121875E61219F980DFB4732BC082C083868234
:20182B000886837A00E4936004A30A80F88683188682121875E493A360051219F980F6D061
:20184B0083D08280B1B4691986017A00E76004090A80F91218758601E7609B1219F90980B4
:20186B00F7F97A01121875E980A8EE601B8FF020F716C002EAC39E500D742030F602743063
:20188B001219F90A80EED002221219A07A03C3E637F60809DAF9E4F5F092E0221219A07A09
:2018AB0003C3E697F60809DAF980EB121998C37A03E633F608DAFA80DD1219987A03C82A18
:2018CB00C8C318E613F6DAFA80CC1219A0AB00A8817F03121B8008AC001219491219ACA8D6
:2018EB00031218C750077863A904121897A803121955600CA8041218B9A80412195570DFA8
:20190B00A80379631219497FFD021B8F1219A0AB00AC011219AC7D19C3A8031218BADD02D8
:20192B00803378631218BA7863A90412196420E7E77863A9041218AAD380DE1219A07A0350
:20194B00E7F60908DAFA221219987A0375F000E6700308DAFA221219A07A03E82AF8E92A37
:20196B00F9181987F0E6B5F006DAF6E4F5F02274FF40F904F5F00422E58124FBF98700129D
:20198B0019AE87000909E7F60809E7F622E58124FBF8860022E58124FBF886011818860010
:2019AB002278637A03760008DAFB22D2AF22C2AF2278FB121B748603088604748075F070FF
:2019CB00121BEB121C4D758921F58DF58B7588597598522278FB121B748682088683E493CD
:2019EB00602D1219F9A380F678FB121B74E63099FDC299F599B40A17740D80F2E430980CE9
:201A0B003098FDC298E599B40D02740A75F0002278FB121B748601E4FBFCFFE709B42D030D
:201A2B000FE709C39430B40A005012FA740A75F000121BAF2AFBE5F03400FC80E4EB8CF047
:201A4B00DF03021C4D2278FB121B748682088683E075F0002278FB121B748682088683E06B
:201A6B00F5F0A3E0C5F02278F9121B74868208868308E6F02278F9121B74868208868308BE
:201A8B00E608F0A3E6F02278FB121B74C293C295D293121B0875F008C3E6139294121AF2FB
:201AAB00D5F0F775F008121AFDA29413D5F0F7C293121B082278FB121B74C293C295D293F3
:201ACB00121B0875F008C308E6139294121AF2D5F0F775F008C318E6139294121AF2D5F04B
:201AEB00F7C293121B0822C295121B08D295121B0822D295121B08C295121B0822C0E07490
:201B0B0005D5E0FDD0E02278FB121B74E63099FDC299F5992274FFF5F030980A3098FDC2B5
:201B2B0098E59975F0002278FB121B74860418188601E4FD121A0BB408028003B47F16ED19
:201B4B0060F21D74081219F974201219F974081219F91980DF1219F9F724F36006090DED00
:201B6B00B504D1E4F7F5F0ED22C82581C822C92581C97A0022D083D082CF2581F581CFC0B6
:201B8B0082C08322CF2581F581CF2229F9E5F03AFA227C00CB30E7011CCB2275F00030E746
:201BAB000215F022FEEBA4FD8EF0ECA4FCEB8EF0A4C5F02C2DC5F022C0F0C0E0E5F06C5486
:201BCB0080FF8CF030F707EB121C4DACF0FBD0E0D0F030F703121C4DBF8005121BEB806281
:201BEB00C002C001AAF0F97E007D007F11C3E933F9EA33FADF08F5F0E9D001D00222ED33B0
:201C0B00FDEE33FEC3ED9BF5F0EE9C40E0ADF0FED380DBBB000122C333C5F033C5F0DBF7B7
:201C2B0022BB000122C3C5F013C5F013DBF722121C3D04700205F022121C4614B4FF021508
:201C4B00F022121C46F4C5F0F4C5F022121CAA4029801E121CAA40227017801E121CAA4029
:201C6B00107017800C121CAA50108005121CBE6009E4F5F022121CBE60F7E4F5F0042212F5
:201C8B001CBE40F680EB121CBE40EF70E480EB121CBE40DD70E480D9121CBE50DD80D2C300
:201CAB009BC5F09C20E70720D207C345F02220D2F9D322C5F0C39C7003E5F09B22FBE493A1
:201CCB00CB22FCE493FB740193CC22FAE493F9740193CA22E31C1E1D0A0A4D696E694C4FD4
:201CEB00474745522056312E3020434F505952494748542028432920313939392C32303068
:201D0B003020574943484954205349524943484F5445000A3E3E000A20696E74657276612D
:201D2B006C2031302D36303020736563203E20002048483A4D4D3A5353203D200020444486
:201D4B002F4D4D2F5952203D20000A253032782F253032782F253032782000253032783A9A
:201D6B00253032783A2530327820002569002575000A2575207265636F72647320617661CA
:201D8B00696C61626C65000A535441525420253032783A25303278203E000A53544F502011
:201DAB0020253032783A25303278203E000A20253032783A2530327820253032783A253052
:201DCB003278000A20535441525420253032783A25303278000A2053544F50202025303207
:201DEB00783A25303278000A2053414D504C494E4720494E54455256414C28736563292071
:201E0B003D202575000A204D414E55414C000A204155544F000A204E6577207265636F72E6
:201E2B00643F28592F4E29000A20253032782F253032782F253032782000253032783A25CA
:201E4B003032783A253032782000256325632F256325632F25632563002C256325633A251B
:201E6B006325633A25632563002C256325632563002C256325632563256325632563000AF8
:201E8B003C2D2D20456E746572206465736372697074696F6E207465787420286D6178202C
:131EAB0035302063686172616374657273292D2D3E0A00B4
:00000001FF
